:020000040000FA
:020000001828BE
:100010002D345234583444343634373436342D3455
:100020002D342D34563430342E34303434342D3491
:100030002010031E20148316FF239000C730810078
:10004000831264008501870183162030850000300B
:1000500087009101831207309900AF2A7B30A100FD
:100060000530A7003328A103A70B3228851E3C28A2
:100070000000A10B362800345D3021020318003443
:1000800008302102031C00340530A7004728A103D3
:10009000A70B4628851A00340000A10B4A28A10AA4
:1000A000851A02340000A10F50280134A700C73080
:1000B000A80064000000A80B5928A70B572800349B
:1000C000153087007B30A70065280000A70B642847
:1000D00000342A3087007B30A7006E280000A70B71
:1000E0006D2800344108430203198528031C8C281D
:1000F000430845020319B12803189928410845020D
:100100000319C128031C7929F9284108450203195C
:10011000F128031CE128D12845084102031941298F
:10012000031C29294308450203195129031C61298D
:1001300011294108C3024307C502602000001430A2
:100140000000C10B9E288700000010300000C30B88
:10015000A4288700000000300000C50BAA288700F3
:1001600090294108C3026020000014300000C10B38
:10017000B4288700000000300000C30BBA288700B5
:1001800090294108C3026020000004300000C10B28
:10019000C4288700000000300000C30BCA28870075
:1001A00090294108C5026020000010300000C10BFA
:1001B000D4288700000000300000C50BDA28870033
:1001C00090294508C1026020000005300000C50BE1
:1001D000E4288700000000300000C10BEA288700F7
:1001E00090296020000000300000C10BF228870039
:1001F00090294108C5024507C30260200000143061
:100200000000C10BFE288700000004300000C50B71
:1002100004298700000000300000C30B0A29870072
:1002200090294308C5024507C10260200000113033
:100230000000C30B16298700000001300000C50B29
:100240001C298700000000300000C10B2229870014
:1002500090294308C1024107C50260200000113007
:100260000000C30B2E298700000010300000C10BD6
:1002700034298700000000300000C50B3A298700B0
:1002800090294308C1026020000011300000C30B18
:1002900044298700000000300000C10B4A29870074
:1002A00090294308C1026020000001300000C30B08
:1002B00054298700000000300000C10B5A29870034
:1002C00090294508C3024307C102602000000530A1
:1002D0000000C50B66298700000001300000C30B39
:1002E0006C298700000000300000C10B72298700D4
:1002F00090294508C1024107C30260200000053073
:100300000000C50B7E298700000004300000C10BEF
:1003100084298700000000300000C30B8A29870071
:10032000420844020319A329031CAA2944084602CF
:100330000319CF290318B729420846020319DF29F8
:10034000031C972A172A4208460203190F2A031C86
:10035000FF29EF294608420203195F2A031C472A96
:100360004408460203196F2A031C7F2A2F2A4208D9
:10037000C4024407C6026920000028300000C20BF6
:10038000BC298700000020300000C40BC229870070
:10039000000000300000C60BC82987000034420866
:1003A000C4026920000028300000C20BD229870057
:1003B000000000300000C40BD82987000034420838
:1003C000C4026920000008300000C20BE229870047
:1003D000000000300000C40BE82987000034420808
:1003E000C6026920000020300000C20BF2298700FD
:1003F000000000300000C60BF829870000344608D2
:10040000C202692000000A300000C60B022A8700E1
:10041000000000300000C20B082A87000034692069
:10042000000000300000C20B102A87000034420890
:10043000C6024607C4026920000028300000C20B33
:100440001C2A8700000008300000C60B222A870003
:10045000000000300000C40B282A87000034440844
:10046000C6024607C2026920000022300000C40B09
:10047000342A8700000002300000C60B3A2A8700A9
:10048000000000300000C20B402A870000344408FE
:10049000C2024207C6026920000022300000C40BDD
:1004A0004C2A8700000020300000C20B522A87002F
:1004B000000000300000C60B582A870000344408B2
:1004C000C2026920000022300000C40B622A8700AB
:1004D000000000300000C20B682A87000034440886
:1004E000C2026920000002300000C40B722A87009B
:1004F000000000300000C20B782A87000034460854
:10050000C4024407C202692000000A300000C60B82
:10051000842A8700000002300000C40B8A2A87006A
:10052000000000300000C20B902A8700003446080B
:10053000C2024207C402692000000A300000C60B54
:100540009C2A8700000008300000C20BA22A870006
:10055000000000300000C40BA82A870000342018D7
:10056000C22AA001FA3056207D30BB00BC00BD007D
:10057000BE00BF00C0000A30A4001930A50005303D
:10058000A600D62A0130A500A01CD62A2F08C1003B
:100590003008C2003108C3003208C4003308C50067
:1005A0003408C600722020120530A6006400A7019E
:1005B0000A30A800851EE42A000064000000A7039A
:1005C0000319A80BDA2A2C2BA101A7030319A803EE
:1005D00003192C2B851ADA2AA10FE52A273081006E
:1005E0006400811B2C2B851EF02AA201F72AF82A11
:1005F0002E20FE3E031D2C2B2108A900A20A2E202E
:10060000FE3E031D2C2B2108AA00A20A2E20FE3E2E
:10061000031D2C2B2108AB00A20A2E20FE3E031D39
:10062000232B2108AC00A20A2E20FE3E031D232B03
:100630002108AD00A20A2E20FE3E031D232B210817
:10064000AE00A20A412B013E031D2C2BA01C412B06
:100650002208A3020319412B0530A600A50B312B5C
:10066000C22AA01CD62A3508C1003608C2003708A5
:10067000C3003808C4003908C5003A08C600722013
:10068000D62A29083B07B500B50C2A083C07B60056
:10069000B60C2B083D07B700B70C2C083E07B80076
:1006A000B80C2D083F07B900B90C2E084007BA0056
:1006B000BA0C3508C1003608C2003708C300380834
:1006C000C4003908C5003A08C600A01C7F2B201AB8
:1006D0007E2B5B30A0193B02A01D4302031C732B31
:1006E0000530A600772BA60B772B20167F2BA019A1
:1006F0007C2B3108C3007E2B2F08C10072202908F3
:10070000BB002A08BC002B08BD002C08BE002D0829
:10071000BF002E08C0001930A500A018B32BA40BF1
:10072000B32B2208A3003508AF003608B000370805
:10073000B1003808B2003908B3003A08B400A01478
:100740005B302F02031CAA2B9E302F02031CAC2B04
:100750003A30AF00A015B22B5B303102031CB22B34
:080760003A30B1002016D62A40
:02400E00DC3F95
:00000001FF
